:10000000F600FFFFFFFFFFFFFFFFFFFFFFFFFFFF08
:10002000FFFFFFFF350DFFFFFFFF6A0EFFFFFFFF22
:10003000FFFFFFFF8813FFFFFFFFFFFFFFFFFFFF33
:100080007E00000000CC23BAC37D94FE73A5E6FF7A
:1000900000080000000A00A00003000000000000AB
:1000A000000000000002070E150000000028333990
:1000B00040464C52565A5F646A6F74797E83898FCA
:1000C00094999DA1A5A8ABAEB1B4B7BA6352431F32
:1000D000006352442E1B4D34210B0052372A1E1B45
:1000E0004E3E3020004E3E302010000000FFFFFF4B
:1000F000FFFFFF00000061D0EE1C1EFE9AB305104A
:1001000000000300FC161FFEA3C0A100BB8BFD1660
:100110009000148AFCC6EAAC00AD0687958684FA86
:10012000F41602FCC6EA8AFCAD06A1009786FAF432
:1001300016800014A6FCC6EA8000AD06879586846A
:10014000FAF416A6FCC6EAA6FCAD06A1009786FA4C
:10015000F49AC501FAFE4D00AD1AB3D289BA61FC1A
:100160002530253083B92583B983B82583B88BEE34
:1001700099BAC2B2AF83B85EBC83B883B95EBD839F
:10018000B9305EBA305EBB99BAAF1020FE0302FCF4
:10019000100CFC0304FCA1009E06FC9E07FCA10CB5
:1001A0009E08FCA1019E09FC419E0AFC0A027B1EDE
:1001B0001002FC9A0E199A42194252BD039A3A193A
:1001C0007A1E0B02AF9AD50DA1059E2EFCA1009EB2
:1001D0006EFCA1209E71FC9AD90A9AA2149AAC02D4
:1001E000311384161B84AC84059AF002FA0C310397
:1001F00084059A840BFA039AFF017110FADCAF9A16
:100200007B049A12058C00191492FC854D00AD11E7
:10021000A100958E16FC9E71FC9A42159A4010FA28
:1002200025310300211492FC8551AD1AA101958E50
:1002300071FC9E16FCA1009E71FC9A42159A8005E5
:100240009A58109AAC108E7BFC4D00BD14148CFC97
:100250008541954814FC8D06A100959A6D0E9A99DA
:100260000E148EFC854195488FFC8D06A100959A51
:10027000C7101490FC8541954891FC8D06A100950E
:100280009A6610148DFC8541954815FC8D06A100D9
:10029000959A2A03148AFC854195488BFC8D06A10A
:1002A00000959A030731230C021B0CAF31738405B0
:1002B0007B849A4010AC0C07A101482EFC8D039A58
:1002C0008005314384054B849AE806315384055BED
:1002D000849A0815316384056B849A42153103852D
:1002E000050B859AD90A311385051B859A9211AFA2
:1002F000AC010B31030332BC012F3A84FA2B9ADD97
:10030000129ABE059A4C179A63173133840AA100DA
:100310009E76FC9AE806FA039A00069ADD129AA6DF
:10032000149AD90A9A96142A84AF8C03039BD80393
:100330008C0018CC010E8E18FC41AD141418FC85ED
:100340004195FA0CA1009E18FCFA05A1009E18FC2C
:10035000A1009E1AFC9E19FCBC010E8E17FC41AD3B
:100360000D1417FC854195FA05A1009E17FCCC01E0
:100370002E3133012A8E18FC51BD07A1029E15FCB7
:10038000FA538E18FC4D05BD059A1406FA478E18CF
:10039000FC4D288D409A1406A1209E15FCFA36319A
:1003A00043012DBC012A8E17FC51BD07A1029E15E9
:1003B000FCFA228E17FC4D05BD059A7506FA168EBD
:1003C00017FC4D288D0F9A7506A1209E15FCFA0585
:1003D000A1029E15FC9B7A04310300039B7A04A1C1
:1003E000009E18FC9E17FCCC010E8E1AFC41AD0D30
:1003F000141AFC854195FA05A1009E1AFCBC010E59
:100400008E19FC41AD0D1419FC854195FA05A1002A
:100410009E19FCCC012E3133012A8E1AFC51BD07E6
:10042000A1029E15FCFA538E1AFC4D05BD059AE7F4
:1004300014FA478E1AFC4D288D409AE714A1209E8D
:1004400015FCFA363143012DBC012A8E19FC51BD31
:1004500007A1029E15FCFA228E19FC4D05BD059AD6
:10046000F714FA168E19FC4D288D0F9AF714A12057
:100470009E15FCFA05A1029E15FCAF9C02658E1B21
:10048000FC41AD06141BFC8541958E93FC4D00BDCF
:10049000268E1BFC4884FC8D1EA1019E93FC8E7150
:1004A000FC310F11146FFC856D08950B0C710B2C32
:1004B0000A0C710A2CFA5A8E93FC51BD548E1BFC07
:1004C0004885FC8D4CA1029E93FC8E71FC310F413E
:1004D000146FFC856D02950B0C710B2C0A0C710AC4
:1004E0002CFA2E8E93FC51BD208E71FC310F13140B
:1004F0006FFC856D01950B0C710B2C0A0C710A2C8D
:10050000FA071470FC856D0195A1009E1BFC9E935B
:10051000FCAF8E70FC311F02FA0B8E70FC310F05A0
:10052000712B212B01AC01528E1CFC4D029D081435
:100530001CFC854195FA48A1009E6FFC9E70FC9EB4
:1005400075FC9A5810A1009E71FCA1079E73FC9A3D
:10055000D90A6A84147BFC854D00AD06A100959AEA
:100560009211A1009E5CFC0A0C710A2C712A212AAE
:10057000017A1EA1039E93FCFA05A1009E1CFCAF0C
:10058000B7312385101477FCB5A0009AFD17B0424F
:1005900052BD022B85B6AF9A970D9A840D9A9D0D88
:1005A0009A55149A620D9AC20D9A100E9A3D0E9A9F
:1005B000E60DAF7B1E13F0049A97057A1EAFA133A8
:1005C0009E6CFCA1079E73FCA1109E84FCA1649EFE
:1005D00085FCAFB7B1B1891CD6A100BE01AE014DFB
:1005E00020AD1772B716AC00AAB64902BD05AE0120
:1005F00072FA09AE0141BE01FAE3A217B0B0B6AF7C
:10060000A000B1A0509AEA11B03270329AD30562BC
:100610009E76FCAF146FFC856D40958E71FC310F9A
:100620000A0B0C710B2C0A0C710A2C8E76FC4D1FD8
:10063000AD428E71FC317E29A1014876FC8D0914F2
:1006400076FC850D0295FA1FA1044876FC8D0914ED
:1006500076FC850D0495FA0F1476FC850D0595FA48
:10066000061476FC854195A11F4876FC9D039E7675
:10067000FC9AE806AF146FFC856D40958E71FC31D5
:100680000F0A0B0C710B2C0A0C710A2C8E76FC4D88
:1006900000AD548E71FC317E398E76FC4D0B8D0988
:1006A0001476FC851D0595FA2F8E76FC4D068D0976
:1006B0001476FC851D0495FA1F8E76FC4D05BD0948
:1006C0001476FC851D0395FA0F1476FC851D0495A0
:1006D000FA061476FC855195A17F4876FC9D05A10C
:1006E000009E76FC9AE806AFB78E76FC5D1F72B767
:1006F00016AC00AAB676B7A000B1A0509A9112B07D
:10070000B0B6AFB78E2EFC9E2FFC023EFC0340FC21
:10071000023CFC033EFC023AFC033CFC0238FC03B6
:100720003AFC0236FC0338FC0234FC0336FC02328D
:10073000FC0334FC0230FC3061013027D20232FC71
:1007400030081EFC30281FFCCA05006143BD033081
:1007500061429D280230FC3061013027D20232FC18
:1007600030081EFC30281FFCDA0500614BBD033049
:10077000614A9D080230FC0332FCFA130230FC305F
:10078000081EFC30281FFC21253025300332FC02D6
:100790001EFC0330FC0240FC30083EFC30283FFCCD
:1007A00030083CFC30283DFC30083AFC30283BFC4B
:1007B000300838FC302839FC300836FC302837FC4B
:1007C000300834FC302835FC300832FC302833FC4B
:1007D000A20831820320FC8C000DA1009E42FCA0E7
:1007E000000344FC9BBB081442FC85419551BD03AA
:1007F0009BBB088E42FC4D02AD039B91080240FC5E
:100800000346FC023EFC4847FCBD04304846FC9DC4
:1008100006023EFC0346FC023CFC4847FCBD04309B
:100820004846FC9D06023CFC0346FC023AFC484755
:10083000FCBD04304846FC9D06023AFC0346FC021F
:1008400038FC4847FCBD04304846FC9D060238FC95
:100850000346FC0236FC4847FCBD04304846FC9D7C
:10086000060236FC0346FC0234FC4847FCBD04305B
:100870004846FC9D060234FC0346FC0232FC484715
:10088000FCBD04304846FC9D320232FC0346FCFAB3
:100890002A8E42FC4D7F9D1D0220FC301846FC3004
:1008A0003847FC0344FCEA00808D10AD0E100000B8
:1008B0000344FCFA061442FC8551950220FC3018D2
:1008C00044FC303845FC4825FCBD04304824FC8DF0
:1008D00006AD04A605FA720220FC301844FC30383C
:1008E00045FC4827FCBD04304826FC8D06AD04A617
:1008F00004FA560220FC301844FC303845FC4829E4
:10090000FCBD04304828FC8D06AD04A603FA3A026B
:1009100020FC301844FC303845FC482BFCBD04302A
:10092000482AFC8D06AD04A602FA1E0220FC3018EF
:1009300044FC303845FC482DFCBD0430482CFC8D6F
:1009400006AD04A601FA02A6008E48FC614EAD0B6E
:10095000A1009E49FC669E48FCFA5C1449FC854156
:10096000958E94FC4D1E9D181494FC854195A10A0A
:100970004849FC9D42A1009E49FC669E2EFCFA3728
:10098000A1194849FC9D30A1009E49FCBC031C8E66
:100990002EFC614E9D06142EFC85419566482EFC6A
:1009A000AD154D00BD119E2EFCFA0C66482EFC9D27
:1009B00006142EFC8551958E2EFC4D00AD2C4D0558
:1009C000AD214D04AD164D03AD0B4D02BD23A1036A
:1009D0009E72FCFA21A1079E72FCFA1AA10B9E726C
:1009E000FCFA13A10F9E72FCFA0CA1009E72FCFA95
:1009F00005A1019E72FC9A010A9A330A9A6C0DB6FF
:100A0000AFA102482FFC9D11482EFC8D0CA010B107
:100A100070B1A0829A9112B0B0A103482FFC8D1240
:100A2000482EFC9D0DA000B1A002B1A0829A9112A7
:100A3000B0B0AF8E2EFC51BD221495FC854D00BD8B
:100A40001AA10295146FFC856D20958E71FC310FF3
:100A50000A0B0C710B2C0A0C710A2C8E71FC311FC5
:100A60004D8E2EFC4D00BD461495FC854D00BD1CE1
:100A7000A10395146FFC856D30958E71FC310F2E9E
:100A80000B0C710B2C0A0C710A2CFA221495FC85A4
:100A90004D02BD1AA10395146FFC856D10958E71E2
:100AA000FC310F0A0B0C710B2C0A0C710A2C8E2EC8
:100AB000FC4D018D0E146FFC855DEF951495FC8542
:100AC0005DFE958E2EFC4D028D0E146FFC855DCF64
:100AD000951495FC855DFC95AFB7B1B1891CD68E98
:100AE00071FC311F2C8E6EFC4D00BD0A10D100BE72
:100AF0000330BE02FA4A8E6EFC4D30BD0A10E5008E
:100B0000BE0330BE02FA3910DB00BE0330BE02FA6B
:100B10002F8E6EFC4D00BD0A10CC00BE0330BE020D
:100B2000FA1E8E6EFC4D30BD0F10E000BE0330BECD
:100B3000021B00711B20FA0810D600BE0330BE0253
:100B4000A100BE01AE014D05AD368E22FCA00030E5
:100B50000D02D2AE0230AE03D48561029D0143AED8
:100B600001A0023188CA24FCD46295638495AE0248
:100B700030AE0380BE0330BE02AE0141BE01FAC4F6
:100B8000B0B0B6AFB7B1891CD68E97FC4D03BD038C
:100B90009B3E0C4D02AD594D01AD314D00AD039B57
:100BA0006E0C9A92149A360E9A630E9A090E7A0176
:100BB0005A016A0113417CA000B1A002B1A0829A3F
:100BC0009112B0B0A1019E97FC9B2F0D8E6EFC4D33
:100BD00030BD07A1029E97FCFA133103000F7B0181
:100BE000A1079E73FC9A4215A1029E97FC9B2F0DB4
:100BF000021EFC5D00EA7F008D05AD039B2F0D02F8
:100C00001EFC5D0030728E9BFC73B762164FFCBBFE
:100C1000B6021EFC5D00D20298FC30610A30612BE6
:100C20000398FC149BFC854D07BD0AA10095A10308
:100C30009E97FCFA06149BFC8541959B2F0D021E86
:100C4000FC5D0030728E9BFC73B7621657FCBBB61E
:100C50008E9BFC4D03BD0E6B01A1009E9BFCA1046D
:100C60009E97FCFA06149BFC8541959B2F0DAC01C9
:100C7000039B2F0D0298FCA208318260BE018E6E8C
:100C8000FC4D30BD16AE011D19BE01C680B1A001DC
:100C90009AFD17B04252BD0313995A8E9AFC49012E
:100CA000AD1AC680B1A0019AFD17B04252BD0D5BCE
:100CB000016A01AE019E9AFC6B015A01021EFC5DA5
:100CC00000EA80009D698E9BFC72B7164FFCAAB6A5
:100CD000720298FC30611A303D000398FC8E9BFC38
:100CE0005D0372B71657FCAAB6728E9BFC73B7628F
:100CF000164FFCBBB68E9BFC72B7164FFCAAB672A1
:100D00000298FC30610A302D000398FC021EFC5D45
:100D10000030728E9BFC5D0373B7621657FCBBB646
:100D20008E9BFC4D079D0341FA02A1009E9BFC9AFD
:100D30006C0DB0B6AFB1B3B589B8B189BAB189BCE1
:100D4000B189BEB17A1E8908A2403182031EFC9A85
:100D50007A0DB099BEB099BCB099BAB099B8B4B296
:100D6000B08F132F03132890132903AF710A2800A3
:100D7000000000717A28710BE6AF710AE6717B28DA
:100D8000710B28AF139F00717AA2710BA013A10001
:100D900013FB00711BA0AFB7F4AC76B6AF13311BD9
:100DA00013200313211F13220A13230F132C0511E1
:100DB0000000110104110200110300110C0113487D
:100DC0000CAF717B43713AE6713BE2138C06134121
:100DD0009B134300AF713BE6717A43AF717B437164
:100DE0003AE6713BE2AF717B6B715AE5715BE113DF
:100DF0006A03F4215D7FF621D8017F11177F136B01
:100E000040AF710A6B717A6BAF717B6B710B6BAF1B
:100E1000717B69714AE5714BE11369281118FF1163
:100E20001900F4215DDFF621D801DFAF111900713F
:100E30000A69717A69AF717B69710B69AF717B6CFB
:100E4000713AE5713BE1136C18111AFF111B00F4A4
:100E5000215DBFF621D801BFAF111B00710A6C7173
:100E60007A6CAF717B6C710B6CAF1A848F31230C71
:100E700012717B6C710B6C6B01717B69710B695B1F
:100E800001FA158C000AA11E9E14FC9A2F0FFA0875
:100E9000A1A09E14FC9ACF0FAF310300108E9CFCD2
:100EA0004D019D09149CFC8541959B2E0FA1009E30
:100EB0009CFCF01B485EFCAD11F01B485EFC9D04E1
:100EC000A101FA02A1FF0E1BF21BC81B00BD0A7193
:100ED0007B6C710B6C6B01FA17C81BFFBD0A6A01B2
:100EE000717B6C710B6CFA086B01710A6C717A6C16
:100EF000F019485FFCAD11F019485FFC9D04A10199
:100F0000FA02A1FF0E19F219C81900BD0A717B6916
:100F1000710B695B01FA17C819FFBD0A5A01717B91
:100F200069710B69FA085B01710A69717A69AFB777
:100F3000A1009E60FC8E2EFC4D028D4DA104187701
:100F4000FC728E2EFC73B716EA00ABB65242AD04AB
:100F500021258AFC9E5EFCA1041877FC728E2EFC73
:100F600073B716F000ABB65242AD0421258AFC9E41
:100F70005FFC3133850C3B858E5EFCF21B8E5FFC83
:100F8000F219A1009E61FCFA44A1009E5EFCF21BD6
:100F90008E61FC4D00BD1AA1041877FC728EF00022
:100FA0005242AD0421258AFCF219F0199E5FFCFA29
:100FB0000F8E61FC4D02BD08111900A1009E5FFC5F
:100FC0001461FC8541954D04BD03A10095B6AF8E1B
:100FD00060FC4D10AD3F4D0CAD3B4D08AD374D04A1
:100FE000AD334D00AD2F4D0EAD0C4D0AAD084D0685
:100FF000AD044D02BD3CA102482EFC9D0CA1289ED3
:101000005EFCA1009E5FFCFA29A1009E5EFCA12867
:101010009E5FFCFA1DA102482EFC9D0CA1059E5E60
:10102000FCA1009E5FFCFA0AA1009E5EFCA1059E49
:101030005FFC1460FC8541954D12BD03A10095AF86
:101040008E62FC4D02AD089A6610A1009E90FC8E47
:1010500075FC5D039E62FCAF8E6EFC4D30AD042BC3
:1010600002FA021B00AF31030002FA3F8E6EFC4D04
:1010700030AD1D8E75FC5D034D02AD0751BD0D2ACF
:1010800002FA2871240201712102FA1F2B02FA1BB5
:101090008E75FC5D034D02AD0751BD0D1A00FA0BB4
:1010A00071140001711100FA021B00AF8E74FC3143
:1010B0000F087B011117059A020EAF8E74FC310FD9
:1010C000059A090E7B01AF8E74FC310E0D9A090E44
:1010D0007B01A1009E5CFC9B9111310300039B915D
:1010E000113136E0043147E00BA1029E5CFC713BFC
:1010F000E0714BE08E74FC311F5C8E5CFC4D00ADEA
:101100005A8E63FC4D05AD074D03AD0351BD077B02
:10111000019A090EFA2B8E77FC4D048D077A019AFD
:10112000090EFA1DA1041877FC61617210FF00AD71
:101130000861FC253025308AF860F2179A020E7B90
:10114000011463FC8541954D20BD46A10095145CBA
:10115000FC855195FA3BA1009E5CFCA1009E63FCBE
:101160008E74FC310F2B8E77FC4D048D077A019A1B
:10117000090EFA1DA1041877FC61617210FF00AD21
:101180000861FC253025308AF860F2179A020E7B40
:1011900001AFB78E7BFC5D03BD1E8E2EFC7216EA7E
:1011A00000AA9E5EFC8E2EFC7216F000AA9E5FFCCA
:1011B000111B7F11197FFA308E7BFC310F0A5A0107
:1011C000717B69710B69FA08717B69710B695B014D
:1011D0008E7BFC311F0A6A01717B6C710B6CFA0803
:1011E000717B6C710B6C6B01B6AFB7B1B1891CD65A
:1011F000711A21710A211B01711B210B01710B2135
:10120000AE02709A0F134252AD0F1B01711B217178
:101210000A21711A21A25AFA74AE08709A0F13713A
:101220001A21710A211B01711B210B01710B21AEC7
:10123000026D01709A0F134252AD0F1B01711B21F9
:10124000710A21711A21A2A5FA43711A21A100BEC7
:1012500001AE014D08AD1B87610197710A21311361
:101260000104876D01970B01710B21AE0141BE0195
:10127000FADF711A21710A21710A210B01710B2108
:101280001B01711B21710A21711A218772B0B0B63E
:10129000AFB7B1B1891CD6711A21710A211B017136
:1012A0001B210B01710B21AE02709A0F134252AD3C
:1012B0000F1B01711B21710A21711A21A2FFFA195A
:1012C000AE08709A0F13AE0A709A0F131B01711BB0
:1012D00021710A21711A21A200B0B0B6AFB7A613CE
:1012E000664D00AD28711A21710A21711A2131133E
:1012F0000110711B211B01711B21710A21711A211F
:10130000FA0B711B210B01710B2156FAD3B6AFB743
:10131000B1B1B1891CD6A100BE03AE034D08AD2406
:10132000AE04317F05711A21FA051B01711B217171
:101330000A21AE046101BE040B01710B21AE034111
:10134000BE03FAD6711A21710A21A100BE01BE02A4
:101350008C011CAE0130AE0280BE0230BE0130EA0C
:1013600010278DECADEA0B01710B21A2FEFA1431AE
:101370001301090B01710B21A2FFFA070B01710B7D
:1013800021A200B0B0B0B6AFB1B3B589B8B189BAD7
:10139000B189BCB189BEB1715AA63146AA06716A3B
:1013A000A69B45143106E30A3107AAF8716AA69B89
:1013B0004514715AA6710BE3F4A5709A7916629ED2
:1013C00067FC3107E331710BE3715AA6F4A54D4A6E
:1013D000BD148E67FC4D17BD0DA1009E71FC9A4295
:1013E000159A0028FADC716AA6F4A570B18E67FC24
:1013F000709A9E15B0FA4E3117AA3E8E67FC709A0D
:101400004216629E69FC3106E3093107AAF8716A47
:10141000A6FA32710BE33146AA05716AA6FA268E46
:1014200069FCF6A53106E3093107AAF8716AA6FA44
:1014300014710BE3716AA6FA0C3107AA05716AA64A
:10144000FA039BC213B099BEB099BCB099BAB099D7
:10145000B8B4B2B08F717BA6710AE7710BE3710B60
:10146000EBF4265DFEF626D806FEF4265DFDF62694
:10147000D806FD13A80813A90013A74A711AAB7167
:101480000AAB714BA6713AA6712AA6710BE7717A65
:10149000A6AF717BA6AFA1009E64FC717AA6716AAB
:1014A000A6AF1399ACAFB7A000B1A0829AEA11B071
:1014B00062765D1C26265DFC72665D03616A9E6D28
:1014C000FC665DE021259E6EFC9A42158E77FC72CB
:1014D000B7169EFCAAB69E6AFC70B1A003B1A082AA
:1014E0009A9112B0B0B6AF8E77FC41AD061477FC7E
:1014F0008541959A0815AF8E77FC4D00AD0614779F
:10150000FC8551959A0815AFB7A1044877FC9D0357
:101510009E77FC8E77FC72B7169EFCAAB6768E6A12
:10152000FC614EAD1B669E6AFCB7A003B1A0829A17
:101530009112B0B02A853A85A1FA9E8CFC9E8EFC51
:10154000B6AFB7A6008E71FC310F06A1066166FA30
:1015500004A10261668E6EFC4D30AD353103003161
:101560008E73FC310F04A14061668E73FC311F0441
:10157000A12061668E73FC312F04A11061663123B6
:101580000307712B212B01FA1331130004A19F6172
:1015900056B7A001B1A0829A9112B0B0B6AFB7B160
:1015A000891CD68730AE06D6A119614E9D039B3F9C
:1015B00016664D108D0BC6A100CA6CFCD46795FA57
:1015C0007E664D088D584D0FAD4C4D0CAD3A4D0B10
:1015D000AD2E4D0AAD204D09AD144D08BD61679E7D
:1015E00074FC67314E041B0CFA551A0CFA51679EB5
:1015F00075FC7A84FA49675D1F9E76FC4A84FA3F3F
:10160000679E77FC5A84FA37679E78FC675D0151C4
:10161000BD2D0A84FA29679E7BFC1A85FA21664D46
:1016200005AD144D07AD0A4D04BD14679E70FCFA5C
:101630000E679E73FCFA08679E71FC6A840A85B087
:10164000B6AFB7D6A100CA6CFCD4859E86FC664DA9
:10165000FFAD1B4D06AD0B4D03BD18A1009E6FFCE9
:10166000FA11BC030E1486FC856D8095FA05A15A0B
:101670009E86FC8E86FC72B6AFB7D6665DF09E87FE
:10168000FC665D0F9E88FCA1804887FC9D05A2FF3B
:101690009B4A178E87FC4D50BD05A2FF9B4A17A1A0
:1016A000304887FC8D51A1104887FC8D238E87FC24
:1016B0004D10BD0FA1024888FC8D3A410888FC728C
:1016C0009B4A17A1024888FC8D2B8E88FC72FA7AFF
:1016D0008E87FC4D20BD0FA1014888FC8D17A10607
:1016E0000888FC72FA64A1014888FC8D5BA1080897
:1016F00088FC72FA55FA51A1604887FC8D258E87C7
:10170000FC4D60BD0FA1034888FC8D3CA10C0888EE
:10171000FC72FA36A1014888FC8D2DA10A0888FCCC
:1017200072FA278E87FC4D70BD0FA1074888FC8D8B
:1017300017A1100888FC72FA11A1014888FC8D08D5
:10174000A1180888FC72FA02A2FFB6AFA001B1A0EE
:10175000509AEA11B062317E074A859A8A01FA02EC
:101760004B85AFB7B1B1891CD6C6CA0300B1A00181
:101770009A9718B062BE01CC8539C6CA0200B1A0E2
:10178000029A9718B0AE0249039D02BE03C6CA0270
:1017900000B1A0039A9718B0AE0249039D02BE03A0
:1017A000C6CA0200B1A0049A9718B0AE0249039DC0
:1017B00002BE03AE014D00BD0CAE039E22FCA10192
:1017C0009E79FCFA0AA1509E22FCA1E09E79FC8E33
:1017D00022FC9E7AFCC6CA0300B1A0009A9718B0FA
:1017E00062BE014D00BD0DA10449038D07AE039EED
:1017F00077FCFA05A1039E77FCB0B0B6AFB7B1B1E4
:10180000891CD6314385497B1E9A92149ADC0D9A25
:101810007A0D0A02AE0830AE09B1AE02709A2619EE
:10182000B062BE014D00AD169AC6189AD218AE0825
:1018300030AE09B1AE02709A2619B062BE010B0239
:101840009A96149AD50D9A6C0D7A1EAE0172FA43CF
:10185000AE0251BD2814A4FC855D0395AE0830AEE0
:1018600009D48570B1AE020D027014A4FC854195B7
:10187000516100B1A0509A9112B0B0FA16AE083082
:10188000AE09D48570B1AE020D0270B1A0509A912C
:1018900012B0B0B0B0B6AFB7B1891CD63143850E27
:1018A000AE0630AE07B187709A1219B0FA15870DDF
:1018B0000270B1A0509AEA11B0AE0630AE07D46201
:1018C00095A200B0B6AF314385059A3E19FA02A23F
:1018D00000AF314385059A3A19FA02A200AF3143AD
:1018E000850D7B1E9A92149ADC0D9A7A0D0A02AF2E
:1018F0003143850D0B029A96149AD50D9A6C0D7A88
:101900001EAF314385059A4219FA02A2FFAF9A46EB
:1019100019AFB7B1891CD6AE0630AE07D4AE0030D1
:101920009A6E1AB0B6AFB7B1891CD6AE0630AE0704
:10193000D4AE00309AC21AB0B6AF9AA81BAF9ABD07
:101940001DAF9A4B1EAFB7B5B19AC5214D00AD057D
:10195000A2F49B671A9A5822A1FF9EB4FCA1009E94
:10196000B5FC9EBDFC8EB5FC9AE820D69AF6204DBB
:1019700000AD5B9A2F214DFFAD0F8EB4FC4DFFBD26
:10198000088EB5FC9EB4FCFA459AEB1F9AFB1F4DDE
:1019900000AD039B531AA1019EBEFC8EB5FC728E56
:1019A000ABFC308EACFC610A309A14204D00AD1BAC
:1019B0008EBEFC519EBEFCBDE2A1019EBDFC8EB55B
:1019C000FC9A9A1F4D00AD039B5A1A9AF31F9A581E
:1019D000228EB5FC4148AFFC9D059EB5FCFA868E73
:1019E000B4FC4DFFBD62A1009EB5FC8EB5FC9AE82B
:1019F00020D69A68214D00BD41B702A8FCD6A1555A
:101A000097869786978697B69AEB1F9AFB1F4D008D
:101A1000BD41C6D48EABFCA3039A63204D00BD0527
:101A20009AF31FFA238EB5FC9A9A1F4D00BD2B9A8C
:101A3000F31F9A5822A1019EBDFC8EB5FC4148AF10
:101A4000FC9D229EB5FCFAA38EBDFC4D00BD12A2EA
:101A500000FA149AF31FA2FEFA0D9AF31FA2FDFAE0
:101A600006A201FA02A2FB9A5822B0B4B6AFB7B5EB
:101A7000B1891CD69A4B224D00AD04A2F3FA3F9ACD
:101A8000921E4DFFAD363087309A4B1FEA0000ADF5
:101A90002780D2AE0230AE03D4C2D6A2006248ADD7
:101AA000FC9D078795868442FAF3665D034D03BD6E
:101AB00003948795A200FA06A2F7FA02A2FAB0B43C
:101AC000B6AFB7B5B1891CD69A4B224D00AD05A271
:101AD000F39BA41B9A921E4DFFBD039B8F1B9EB4CC
:101AE000FC02A8FC3008B1FC302D00D4A1FF959475
:101AF00095949594958772B702A8FCD66297B6AE76
:101B00000230AE03D402A8FCD686A2008597868454
:101B1000426248ADFC8DF502A8FC3008B1FC302DC6
:101B200000DA0100D687A00030978630978EB4FC8B
:101B30009AE8203008B2FC3028B3FC03B8FCA101BD
:101B40009EBEFC8EB4FC9AFE1E03BAFC9AEB1F9A52
:101B5000FB1F4D00BD3D02BAFC48B9FC8D07304863
:101B6000B8FC9D3330D48EB1FC738EABFC9A6320ED
:101B70004D00AD2B4D1EAD098EBEFC51AD1D9EBE60
:101B8000FCC43008B1FC302D008003BAFCFAC7A2B7
:101B9000FAFA11A2FEFA0AA2F5FA06A2F6FA02A2CF
:101BA000009AF31FB0B4B6AFB7B5B19A58229A4BAA
:101BB000224D00AD05A2F39BB61DA1009EBDFC9A6F
:101BC000921E4DFFBD039B9F1D9EB4FC8EB4FC9ED8
:101BD000B5FC9AE82003B6FC8EB5FC4148AFFC8DFD
:101BE00002A10048B4FCBD039BA71D9EB5FC9AE86A
:101BF0002003B8FCD69AF6204D00ADDC8EAAFC314D
:101C00000F509AEB1F9AFB1F4D00AD039BA31DA124
:101C1000019EBEFC8EB5FC728EABFC308EACFC61BE
:101C20000A309A14204D00AD238EBEFC519EBEFC9E
:101C3000BDE28EB5FC9A9A1F4D00AD039BAF1DA16E
:101C4000019EBDFC9AF31F9A5822FA8C9AF31F9AB0
:101C5000582202B8FCD69A68214D00AD039BD81BD0
:101C600002B8FCCA080003BAFCA1009EBEFC8EAEFE
:101C7000FC41308EBEFC61488D039B311D308EB41B
:101C8000FC9A4B1FEA0000BD039B241DD602A8FC52
:101C9000D4A200879586846248B1FC9D0342FAF382
:101CA0009AEB1F9AFB1F4D00AD039BA31DA1019E44
:101CB000BFFC02BAFCD43008B1FC302D005DFC70D2
:101CC00094655DFC614884AD2602A8FCD6A15597B9
:101CD00086978697869702B8FCCA0400D4A3038E21
:101CE000ABFC9A63204D00BD719AF31F9BD81B8EED
:101CF000B1FC738EABFC9A63204D00AD184D1EAD48
:101D0000098EBFFC519EBFFCAD50C43008B1FC3001
:101D10002D0080FAA0C43008B1FC302D008003BA39
:101D2000FC9AF31F8EBEFC419EBEFC9A58229B6E0D
:101D30001C9AEB1F9AFB1F4D00AD02FA6602A8FC2D
:101D4000D6A1559786978697869702B8FCD4A303A9
:101D50008EABFC9A63204D00AD188EB5FC9A9A1F8D
:101D60004D00BD4B9A5822A1019EBDFC9AF31F9BCA
:101D7000D81B02B6FCCA0400D48EABFCA3039A6342
:101D8000204D00AD0F8EB4FC9A9A1F4D00BD20A1CE
:101D9000019EBDFC8EBDFC4D00BD10A200FA14A238
:101DA000FAFA13A2FEFA0CA2F8FA0BA201FA04A2A4
:101DB000FDFA009AF31F9A5822B0B4B6AFB7B5B186
:101DC0009A4B224D00AD04A2F3FA7C9A921E4DFF6D
:101DD000AD649EB4FC73634D00BD048EAFFC7353C1
:101DE0008EB4FC614BAD57639AE820D69AF6204D2D
:101DF00000ADE3639EB5FC9AEB1F9AFB1F4D00BD3F
:101E000039A1019EBEFC8EB5FC728EABFC308EAC4F
:101E1000FC610A309A14204D00AD278EBEFC519E05
:101E2000BEFCBDE28EB5FC9A9A1F4D00AD04A2FD2A
:101E3000FA12A2FCFA0EA2FAFA0DA2FEFA06A2F912
:101E4000FA05A2009AF31FB0B4B6AFB7B5B19A4B7A
:101E5000224D00BD379A921E4DFFAD30729AE82098
:101E6000D6629AFE1ED4C63008B2FC3028B3FC30CD
:101E7000611C30613DD6A0008EB1FC3080D4C6A27A
:101E80000030611C30613D8D0542FAF5A2FFB0B40F
:101E9000B6AFB7A6006648AFFC9D5F9AE82003C0C6
:101EA000FC66A700674D089D167202C0FCB7D6AA53
:101EB000B6726773B702A8FCD662BBB647FAE5B73D
:101EC00002A8FCD6AE0030AE01EA5555BD28868684
:101ED000AE0030AE01EA5555BD1C8686AE0030AE70
:101EE00001EAFFFFBD108686AE0030AE01EAFFFFBB
:101EF000BD04B666FA06B646FA9BA1FFB6AFB79A1E
:101F0000E820D43008B2FC3008B3FCD603C0FCC4CF
:101F1000CA0800D4C63018B1FC303D0090D6614DDF
:101F20008D24BD0530614C8D1DB58EB1FCA00030F7
:101F300090D4C630610C30612DD485B44DFFBD0600
:101F4000C603C0FCFACE02C0FCB6AFB73073309AFD
:101F5000E820D43008B2FC3008B3FCD6C4CA08006C
:101F6000D4C63018B1FC303D0090D6614D8D26BDF1
:101F70000530614C8D1FB58EB1FCA0003090D4C6E9
:101F800030610C30612DD485B44D00BDD487614BD8
:101F9000BDCFC6FA03100000B6AFB79AE820D4024E
:101FA000A8FCD6A100BE00BE01BE02BE03A701A6CA
:101FB00001A3048EABFC9AA9204D00BD04A700FA32
:101FC0000356BDEDC4CA0400D4A601A3048EABFC25
:101FD0009AA9204D00BD04A700FA0356BDED674D38
:101FE00000AD04A1FFFA02A100B6AF7B1E9A002D3E
:101FF0007A1EAF7B1E9A0D2D7A1EAFB3B502A6FCDA
:102000009A1A2D9A7B2E624D00AD04A1FFFA02A10F
:1020100000B4B2AFB7B3B5D69A5822C63072A10099
:10202000A300B37B1E9AB52D7A1E62B24D1BBD1E56
:102030009A5822C63072A100A300B37B1E9A2C2DA1
:102040007A1E62B24D00ADD04D1FADCCFA084D00E6
:10205000AD084D1FADC2A1FFFA02A1009A5822B4EB
:10206000B2B6AFB7B3B59EC4FCC403C2FC632424AC
:102070005D3F4172A3009A582202A8FCD6B7B31064
:10208000C2FC7B1E9A8A2E7A1E62B2B64D00AD103B
:102090004D1FADD94D1EAD04A1FFFA06A11EFA02D7
:1020A000A1009A5822B4B2B6AFB7B3B59EC4FCC46F
:1020B00003C2FC635124245D3F4172A3009A58225D
:1020C00002A8FCD6B7B310C2FC7B1E9A522D7A1E12
:1020D00062B2B64D00AD084D1FADD8A1FFFAC3A145
:1020E000009A5822B4B2B6AFB7728EACFC610AA0A7
:1020F00000212727B6AFB7AE004D00BD12AE014D8F
:1021000000BD0CAE024D00BD06AE034D00AD1CAED1
:10211000044D00BD12AE054D00BD0CAE064D00BD18
:1021200006AE074D00AD04A1FFFA02A100B6AFB79D
:10213000AE004D55BD2EAE014D55BD28AE024D55DC
:10214000BD22AE034D55BD1CAE044DFFBD16AE0500
:102150004DFFBD10AE064DFFBD0AAE074DFFBD04DD
:10216000A100FA02A1FFB6AFB7AE004DFFBD2EAE83
:10217000014DFFBD28AE024DFFBD22AE034DFFBD98
:102180001CAE044DFFBD16AE054DFFBD10AE064D95
:10219000FFBD0AAE074DFFBD04A100FA02A1FFB6C4
:1021A000AFD6AE054D069D1AAE064D399D14AE074D
:1021B0004D018D0E4DFF9D0AAE084DFE9D04A10000
:1021C000FA02A1FFAFB110B4FCD6DAA6FCA10096CA
:1021D0009750BDFBB0D69AA1214DFFAD6DAE00303A
:1021E000AE0103A6FC8686AE0030AE0103A8FC86D5
:1021F00086879EAAFC86879EABFC86879EACFCA148
:10220000049EAFFC86879EADFC86879EAEFC8EAD9D
:10221000FC41A00030A204318240A1043188D49056
:10222000309EB1FC100800A200D630610C30612D48
:10223000EA01049D0342FAF1C603B2FC629EB0FCBF
:102240008EAAFC61FA9EAAFCA100AF8EAAFC317F87
:1022500004A100FA02A1FFAFB18EAAFC311F04A1B4
:10226000ACF699B0AFFFFFFFFFFFFFFFFFFFFFFFDF
:10280000B79A5C287A019A002D1020FE9A1A2D9A08
:1028100087284252AD0A5A019A0D2D716AA6FAFE16
:102820007B01A1009EA2FE7A019AC62862764D0025
:10283000AD106A019A0D2D716AA6711BA013994AF9
:10284000FAFE7B019A4F296276317F089A0D2D712D
:102850006AA6FAFE7B01FACFFAFEB6AF713AA6710C
:102860007B6C710B6C6B01717B69710B695B017126
:102870007B6B710B6B7A01711AA07B1EFEE4FFFF6C
:10288000FEE6FFFF7A1EAFB7A6000A029A7B2E4231
:1028900052AD04A281FA2DA700674D0AAD1F377013
:1028A00037B1A0009AB52DB0624D1BBD0D37703702
:1028B000B1A0009A2C2DB062616647FADC664D002B
:1028C000AD02A282B6AFB7B1B1891CD6710BE3716C
:1028D0005AA63106E3063106AA02FAF63107AA041F
:1028E000A201FA67F4A54D3ABDE29AD82962BE0367
:1028F0009AD82962BE01A0003030B19AD829B030F0
:10290000610A302D0003A0FE9AD82952BD04A2020C
:10291000FA39A100BE02AE0249039D149AD829AE2D
:102920000273B7621690FEBBB6AE0241BE02FAE673
:102930009AD829AE024D109D1072B7A1FF1690FED5
:10294000BAB6AE0241BE02FAEAA200B0B0B6AFB764
:1029500002A0FEEA00288D04A202FA7A5A0116901B
:10296000FEB7A004B110A0FE9A522DB0B04252ADF5
:1029700004A2C1FA616A0102A0FE5DFCA000242449
:102980005D3F30B1709A8F2DB04252AD435B01165E
:1029900090FEB7A004B110A0FE9A522DB0B04252E2
:1029A000AD04A2C2FA3002A0FE99B8EEBA0000EE61
:1029B000BC00C0100F009A7501A10A9A5601F0B828
:1029C00070B1A0009A8F2DB04252AD04A2C3FA0696
:1029D0006B015B01A200B6AFB7710BE3715AA63170
:1029E00006E302FAFAF4A5774D308D0CA139614F58
:1029F0008D06671D3076FA20674D418D0CA15A6116
:102A00004F8D06671D3776FA0F674D618D0AA17AE3
:102A1000614F8D04671D577666262626265DF07663
:102A2000710BE3715AA63106E302FAFAF4A5774D69
:102A3000308D0DA139614F8D07671D306166FA2217
:102A4000674D418D0DA15A614F8D07671D37616636
:102A5000FA10674D618D0BA17A614F8D05671D5787
:102A60006166367236B6AFFFFFFFFFFFFFFFFFFF65
:102D000013C0A513C40113C4FE13C401AF13C0A59F
:102D100013C40013C4FF13C400AF22B161F8B6A2FC
:102D2000009A0081A109BE13BE1423AFB7D2891C3B
:102D3000D6AE0473629AC72EAD1122B161F8B0BE4F
:102D400003A2039A008123F0E3FA02A10572A30013
:102D5000B6AFB7D4891CD6AE0473AE0630AE07D674
:102D6000C49AE62EAD2222B1B3B761F8B0BE0560B9
:102D7000BE04B0BE0360BE00B0BE0260BE01A204CD
:102D80009A008123F0E3FA02A10572A300B6AFB75F
:102D9000D2891CD6AE0473629AC72EAD1122B161DE
:102DA000F8B0BE03A2069A008123F0E3FA02A1055F
:102DB00072A300B6AFB7D2891CD6AE0473629AC7AD
:102DC0002EAD1122B161F8B0BE03A2089A00812392
:102DD000F0E3FA02A10572A300B6AFB7D2891CD600
:102DE000AE0430AE05E2D6C2D4AE004D05BD1870BB
:102DF000AE0273AE019AC72EAD153022B5B161F89F
:102E0000B030BE0060FA124D03AD084D04AD04A110
:102E100005FA4722B5B161F8B0BE03B0BE0560BE89
:102E200004A2099A0081234D05BD2D634D00AD28F4
:102E3000324D208D234D309D1F62E4D6AE0170AE21
:102E400002E4BE02A0002626262626273027E430EC
:102E5000611C30613D60BE01F0E372A300B6AF605B
:102E6000B12261F8891CCA0200BE0560BE04A20A34
:102E70009A008123B0F0E372A300AF2261F8A20EA2
:102E80009A008123F0E372A300AFB7D4891CD6AEB9
:102E90000473AE0630AE07D6C49AE62EAD2222B138
:102EA000B3B761F8B0BE0560BE04B0BE0360BE003B
:102EB000B0BE0260BE01A2179A008123F0E3FA02BD
:102EC000A10572A300B6AF334D208D174D309D1371
:102ED00033724D069D0B26262626610B323332FABD
:102EE00002A1FF4DFFAFB7D6AE0070AE01EA008081
:102EF0008D25EA00C09D20753072A000AE024D06FF
:102F00009D10262626262627302730610D302D00DD
:102F1000FA0910FFFFFA043072A100B6EAFFFFAF12
:00000001FF
